:100000000C947B000C948D000C948D000C948D004E
:100010000C948D000C948D000C948D000C948D002C
:100020000C948D000C948D000C948D000C94B500F4
:100030000C94DA000C948D000C948D000C948D00BF
:100040000C948D000C948D000C948D000C948D00FC
:100050000C948D000C948D000C948D000C948D00EC
:100060000C948D000C948D000C948D000C948D00DC
:100070000C948D0000010000E0001200020000CE90
:10008000001200030000CA000401030904BC000CB4
:1000900002030904AC000E030309049E000C0C03C8
:1000A0005B007300650072005D0000000E035B00E2
:1000B000700072006F0064005D0000000C035B00C4
:1000C0006D00660067005D0000000403090409027A
:1000D0001200010100C0320904000000FF0101000C
:1000E0001201000000000040CDAB03F0CDAB0102D7
:1000F00003010000000011241FBECFEFD2E0DEBFDD
:10010000CDBF21E0A0E0B1E001C01D92A534B2074F
:10011000E1F70E9495050C94B4050C9400008091C1
:10012000E80080FFFCCF08958091E80082FFFCCFBB
:100130000895E1E6F0E080E88083108208958FEF73
:100140008093440180EA8093D8001092630086E097
:1001500089BD09B400FEFDCF80E88093D8001092DD
:10016000E0008CE08093E20008951F920F920FB69A
:100170000F9211248F939F938091E1001092E100E0
:1001800083FF11C01092E90081E08093EB00109290
:10019000EC0092E39093ED0098E09093F0001092C1
:1001A0000301809344019F918F910F900FBE0F9098
:1001B0001F9018951F920F920FB60F9211242F9235
:1001C0003F92EF92FF920F931F932F933F934F9382
:1001D0005F936F937F938F939F93AF93BF93CF93CF
:1001E000DF93EF93FF931092E9008091E80083FF83
:1001F00080C49091F1008091F100C091F1002091B4
:10020000F100D0E0D22B2091F1004091F10000915B
:10021000F1003091F10010E0132B32EF3093E80041
:10022000863009F047C030E0342B46E084E790E0A8
:10023000FC01659174916C177D0739F4FC013296CD
:10024000659174916217730721F00796415081F709
:1002500050C4FC01349625913491FC01369684916A
:10026000E8010F3F110519F010F0CFEFD0E0C817EB
:1002700008F48C2F5EEF9091E800492F4570D9F378
:1002800092FD3AC4982F813408F090E4F901492F87
:10029000442331F064916093F10041503196F8CFDE
:1002A000290F311D891B5093E8008111E4CF903450
:1002B00011F322C4853049F48EEF8093E8000E9448
:1002C0008F00C068C093E30017C4893071F59111A5
:1002D00010C4C09303018EEF8093E80041E082EFE9
:1002E00090E04093E9009C012F5F3F4FFC01549147
:1002F0005093EB00552359F0F90124912093EC0021
:100300009C012D5F3F4F319684918093ED004F5FAC
:10031000453011F0C901E5CF8EE18093EA001092DB
:10032000EA0082E080934401E7C3883041F49038CA
:1003300009F0DFC30E948F008091030131C0811159
:1003400007C00E948F001092F1001092F100CDC3FF
:10035000833A81F48091E800982F9570D9F382FD5B
:10036000CBC38BE08093F1008150E1F78EEF809357
:10037000E800BFC3843AB9F40E948F0034E03093A0
:10038000F10025E02093F10096E09093F10087E0E2
:100390008093F1003093F1002093F1009093F100ED
:1003A0008093F100A2C3863A39F580E890E06EEFC1
:1003B0002091E800322F3570D9F322FD9DC39C01B6
:1003C0008134910510F020E430E0422F442351F0B5
:1003D0005091020171E0750F709302015093F1008A
:1003E0004150F4CF821B930B6093E800009701F714
:1003F00020343105E9F280C3853A09F07AC30E94BE
:100400009400519A59987801FFE3EF22FF24E80104
:1004100066E0D695C7956A95E1F70BEF84E191E028
:100420001FE2180F209709F44BC39091F1009093AD
:10043000040150E8252E2220D1F0822D8923599ADB
:1004400061F02694000000000000000000000000A1
:10045000000000000000599808C0000000000000E3
:10046000599826940000000000000000E4CF90910D
:10047000F100909305018091F10080930601809135
:10048000F100809307018091F1008093080140E81A
:10049000242E2220D1F0822D8923599A61F02694AE
:1004A000000000000000000000000000000000004C
:1004B0000000599808C000000000000059982694D8
:1004C0000000000000000000E4CF8091F100809364
:1004D00009018091F10080930A018091F1008093DD
:1004E0000B018091F10080930C0130E8232E909154
:1004F00006012220D1F0822D8923599A61F0269499
:1005000000000000000000000000000000000000EB
:100510000000599808C00000000000005998269477
:100520000000000000000000E4CF8091F100809303
:100530000D018091F10080930E018091F100809374
:100540000F018091F1008093100120E8222E9091FC
:1005500007012220D1F0822D8923599A61F0269437
:10056000000000000000000000000000000000008B
:100570000000599808C00000000000005998269417
:100580000000000000000000E4CF8091F1008093A3
:1005900011018091F100809312018091F10080930C
:1005A00013018091F100809314018091F1008093F8
:1005B000150190E8292E909108012220D1F0822D7A
:1005C0008923599A61F02694000000000000000081
:1005D00000000000000000000000599808C0000062
:1005E0000000000059982694000000000000000060
:1005F000E4CF8091F100809316018091F100809307
:1006000017018091F100809318018091F10080938F
:10061000190180E8282E909109012220D1F0822D25
:100620008923599A61F02694000000000000000020
:1006300000000000000000000000599808C0000001
:1006400000000000599826940000000000000000FF
:10065000E4CF8091F10080931A018091F1008093A2
:100660001B018091F10080931C01B0E82B2E90912A
:100670000A012220D1F0822D8923599A61F0269413
:10068000000000000000000000000000000000006A
:100690000000599808C000000000000059982694F6
:1006A0000000000000000000E4CF8091F100809382
:1006B0001D018091F10080931E018091F1008093D3
:1006C0001F01A0E82A2E90910B012220D1F0822D4B
:1006D0008923599A61F02694000000000000000070
:1006E00000000000000000000000599808C0000051
:1006F000000000005998269400000000000000004F
:10070000E4CF8091F100809320018091F1008093EB
:1007100021018091F100809322018091F10080936A
:100720002301F0E82F2E90910C012220D1F0822D90
:100730008923599A61F0269400000000000000000F
:1007400000000000000000000000599808C00000F0
:1007500000000000599826940000000000000000EE
:10076000E4CF8091F100809324018091F100809387
:1007700025018091F100809326018091F100809302
:100780002701E0E82E2E90910D012220D1F0822D3C
:100790008923599A61F026940000000000000000AF
:1007A00000000000000000000000599808C0000090
:1007B000000000005998269400000000000000008E
:1007C000E4CF8091F100809328018091F100809323
:1007D00029018091F10080932A018091F10080939A
:1007E0002B0170E8272E90910E012220D1F0822D4E
:1007F0008923599A61F0269400000000000000004F
:1008000000000000000000000000599808C000002F
:10081000000000005998269400000000000000002D
:10082000E4CF8091F10080932C018091F1008093BE
:100830002D018091F10080932E018091F100809331
:100840002F0160E8262E90910F012220D1F0822DF9
:100850008923599A61F026940000000000000000EE
:1008600000000000000000000000599808C00000CF
:1008700000000000599826940000000000000000CD
:10088000E4CF8091F100809330018091F10080935A
:1008900031018091F100809332018091F1008093C9
:1008A000330150E8252E909110012220D1F0822DA5
:1008B0008923599A61F0269400000000000000008E
:1008C00000000000000000000000599808C000006F
:1008D000000000005998269400000000000000006D
:1008E000E4CF8091F100809334018091F1008093F6
:1008F00035018091F100809336018091F100809361
:10090000370140E8242E909111012220D1F0822D50
:100910008923599A61F0269400000000000000002D
:1009200000000000000000000000599808C000000E
:10093000000000005998269400000000000000000C
:10094000E4CF8091F100809338018091F100809391
:1009500039018091F10080933A018091F1008093F8
:100960003B0130E8232E909112012220D1F0822DFC
:100970008923599A61F026940000000000000000CD
:1009800000000000000000000000599808C00000AE
:1009900000000000599826940000000000000000AC
:1009A000E4CF8091F10080933C018091F10080932D
:1009B0003D018091F10080933E018091F100809390
:1009C0003F0120E8222E909113012220D1F0822DA8
:1009D0008923599A61F0269400000000000000006D
:1009E00000000000000000000000599808C000004E
:1009F000000000005998269400000000000000004C
:100A0000E4CF8091F100809340018091F1008093C8
:100A100041018091F100809342018091F100809327
:100A20004301C130D10511F00093E800E4E1F1E0A9
:100A300090E8292E91912220D1F0822D8923599A74
:100A400061F026940000000000000000000000009B
:100A5000000000000000599808C0000000000000DD
:100A6000599826940000000000000000E4CF1E13F7
:100A7000DFCFC130D10511F00E94940080E8282E0C
:100A8000909143012220D1F0822D8923599A61F05F
:100A9000269400000000000000000000000000009C
:100AA00000000000599808C000000000000059989C
:100AB00026940000000000000000E4CF2197B2CC93
:100AC000E114F10429F08BEF8093E8000E94940078
:100AD000599880E090E08E159F0521F02091F1005B
:100AE0000196F9CF8BEF8093E8008EEF8093E800BA
:100AF00003C081E28093EB00FF91EF91DF91CF91F2
:100B0000BF91AF919F918F917F916F915F914F9125
:100B10003F912F911F910F91FF90EF903F902F9059
:100B20000F900FBE0F901F901895F89481E08AB92E
:100B30000E9499000E949F0078942FEF89E698E127
:100B4000215080409040E1F700C000002FEF89E67F
:100B500098E1215080409040E1F700C00000809172
:0C0B600044018230E4F3FFCFF894FFCF93
:00000001FF
